:100000000C9463000C948B000C948B000C948B006C
:100010000C948B000C948B000C948B000C948B0034
:100020000C948B000C948B000C948B000C948B0024
:100030000C948B000C948B000C948B000C948B0014
:100040000C94A2050C948B000C9436070C948B0036
:100050000C948B000C948B000C948B000C948B00F4
:100060000C948B000C948B000000000024002700EF
:100070002A0000000000250028002B0000000000DE
:1000800023002600290004040404040404040202DA
:100090000202020203030303030301020408102007
:1000A0004080010204081020010204081020000012
:1000B0000007000201000003040600000000000029
:1000C00000008D00320811241FBECFEFD4E0DEBF48
:1000D000CDBF11E0A0E0B1E0EEE2FAE102C0059090
:1000E0000D92A233B107D9F712E0A2E3B1E001C04B
:1000F0001D92A934B107E1F710E0C6ECD0E004C0CE
:100100002297FE010E94110DC23CD107C9F70E943F
:100110006C080C94150D0C940000CF92EF920F9385
:1001200082E391E06CE04BE025E004E053E0E52E53
:1001300032E0C32E0E946D056091080170910901A3
:1001400080910A0190910B0127E93CE041EB5EE3CD
:100150000E940A0C6093590170935A0180935B01CD
:1001600090935C0160910C0170910D0180910E01E2
:1001700090910F0122E831EF4EEB5DE30E940A0CF3
:1001800060935D0170935E0180935F0190936001C5
:100190000F91EF90CF9008952F923F924F925F92E0
:1001A0006F927F928F929F92AF92BF92CF92DF9287
:1001B000EF92FF920F931F93CF93DF93C0E0D0E0B5
:1001C0002AC18091650190916601909362018093AC
:1001D000610180916701909168019093640180931F
:1001E0006301809104010E949606909366018093BA
:1001F0006501809106010E9496067C01909368013A
:10020000809367016090710170907201809073011A
:10021000909074016092690170926A0180926B0102
:1002200090926C012090750130907601409077019A
:100230005090780120926D0130926E0140926F01D2
:10024000509270016091650170916601882777FD79
:100250008095982F0E945A0B9B01AC01C401B301F9
:100260000E94570A5B016C0160916101709162010B
:10027000882777FD8095982F0E945A0B9B01AC012F
:10028000C601B5010E94560A2BED39EF4EE75FE338
:100290000E940A0C5B016C01609371017093720102
:1002A00080937301909374010027F7FC0095102F41
:1002B000C801B7010E945A0B9B01AC01C201B101F8
:1002C0000E94570A7B018C01609163017091640167
:1002D000882777FD8095982F0E945A0B9B01AC01CF
:1002E000C801B7010E94560A2BED39EF4EE75FE3D4
:1002F0000E940A0C7B018C0160937501709376015A
:100300008093770190937801C601B501A401930110
:100310000E94560A20911001309111014091120162
:10032000509113010E940A0C9B01AC01C401B3015E
:100330000E94570A3B014C016093790170937A0146
:1003400080937B0190937C01C601B501A6019501C4
:100350000E940A0C9B01AC016093810170938201A1
:10036000809383019093840160918D0170918E013F
:1003700080918F01909190010E94570A60938D01A6
:1003800070938E0180938F0190939001C801B70103
:10039000A80197010E940A0C9B01AC0160937D01AA
:1003A00070937E0180937F01909380016091890119
:1003B00070918A0180918B0190918C010E94570A63
:1003C0006093890170938A0180938B0190938C01D3
:1003D000C401B301A80197010E940A0C9B01AC0162
:1003E00060938501709386018093870190938801C3
:1003F000609191017091920180919301909194018B
:100400000E94570A60939101709392018093930127
:100410009093940121962091020130910301C2171B
:10042000D3070CF4CECEB901882777FD8095982F9D
:100430000E945A0B7B018C0160918D0170918E019D
:1004400080918F0190919001A80197010E94BF0AAD
:100450000E94710C9B01AC016091590170915A018D
:1004600080915B0190915C010E940A0C6093A10154
:100470007093A2018093A3019093A40160918901DC
:1004800070918A0180918B0190918C01A801970154
:100490000E94BF0A0E94710C9B01AC0160915D013A
:1004A00070915E0180915F01909160010E940A0C41
:1004B0006093A5017093A6018093A7019093A80172
:1004C0008091490190914A01A0914B01B0914C015A
:1004D0008093450190934601A0934701B093480152
:1004E0000E94EA055B016C016093490170934A0127
:1004F00080934B0190934C0180914501909146016E
:10050000A0914701B0914801A6019501281B390B24
:100510004A0B5B0B20934D0130934E0140934F01EA
:10052000509350016091590170915A0180915B0183
:1005300090915C0120915D0130915E0140915F01DD
:10054000509160010E940A0C20919101309192011A
:1005500040919301509194010E940A0C7B018C01FF
:100560006091020170910301882777FD8095982F93
:100570000E945A0B9B01AC01C801B7010E94BF0A3F
:100580007B018C0160939501709396018093970194
:10059000909398016091A1017091A2018091A301B3
:1005A0009091A4012091A5013091A6014091A7014D
:1005B0005091A8010E940A0C9B01AC016093990123
:1005C00070939A0180939B0190939C01C801B7019D
:1005D0000E94BF0A60939D0170939E0180939F01CA
:1005E0009093A001E0925501F092560100935701BB
:1005F000109358018091510190915201A0915301A3
:10060000B0915401A6019501281B390B4A0B5B0BD5
:10061000DA01C90181509C45A642B54040F0A09244
:100620005101B0925201C0925301D092540186E31D
:1006300092E00E94C407892BA1F064E670E080E09C
:1006400090E00E94F80582E391E00E94AF0409C0A7
:1006500086E392E00E94EF07682F82E391E00E9418
:100660009D0486E392E00E94C4071816190684F3DD
:100670004091950150919601609197017091980178
:1006800086E392E022E030E00E94480A86E392E0AE
:1006900060E240E050E00E94910940919901509140
:1006A0009A0160919B0170919C0186E392E022E0A7
:1006B00030E00E94480A86E392E060E240E050E0C9
:1006C0000E94910940919D0150919E0160919F016E
:1006D0007091A00186E392E022E030E00E94480A97
:1006E00086E392E060E240E050E00E949109409190
:1006F000A1015091A2016091A3017091A40186E330
:1007000092E022E030E00E94480A86E392E060E254
:1007100040E050E00E9491094091A5015091A6014E
:100720006091A7017091A80186E392E022E030E099
:100730000E944B0A4091550150915601609157011A
:100740007091580186E392E022E030E00E944B0A6B
:1007500080E090E0A0E0B0E080938D0190938E0166
:10076000A0938F01B09390018093890190938A01A7
:10077000A0938B01B0938C0180939101909392018F
:10078000A0939301B0939401DF91CF911F910F91AA
:10079000FF90EF90DF90CF90BF90AF909F908F90A1
:1007A0007F906F905F904F903F902F90089586E3D9
:1007B00092E040E855E260E070E00E94670782E363
:1007C00091E060E142E020E00E94B70408950F93B9
:1007D0001F938C01FC01848160E00E94DE0681E0B1
:1007E00090E00E945106F801848161E00E94DE06DB
:1007F00081E090E00E945106F801848160E00E944F
:10080000DE0684E690E00E9451061F910F91089544
:10081000CF92DF92EF92FF920F931F93CF93DF93CC
:10082000D82EC92E282F392FC9018C01C0E0D0E065
:10083000E62EFF24F801858161E00E94B806B70129
:100840000C2E02C0759567950A94E2F76170F80165
:1008500085810E94DE0621960F5F1F4FC830D105AB
:1008600049F78D2D9C2D0E94E703DF91CF911F91B9
:100870000F91FF90EF90DF90CF900895CF92DF928D
:10088000EF92FF920F931F93CF93DF93D82EC92E31
:10089000282F392FC9018C01C0E0D0E0E62EFF24BB
:1008A000F801858161E00E94B806B7010C2E02C0F4
:1008B000759567950A94E2F76170F80185810E9449
:1008C000DE0621960F5F1F4FC430D10549F78D2DED
:1008D0009C2D0E94E703DF91CF911F910F91FF9014
:1008E000EF90DF90CF9008951F93CF93DF93EC01AB
:1008F000162F8A81642F0E94DE068B818F3F19F0AC
:1009000060E00E94DE068D8584FF05C0CE01612F68
:100910000E9408040EC0612F70E084E07595679511
:100920008A95E1F7CE010E943E04CE01612F0E941C
:100930003E04DF91CF911F91089541E00E9474041D
:10094000089540E00E9474040895FC016685862F96
:10095000846086876C60CF010E94A104089561E0E5
:100960000E94A10480ED97E00E9451060895CF9364
:10097000DF93EC01423018F08D8588608D87498BBC
:100980001A8A222329F0413019F48D8584608D87DD
:1009900080E593EC0E9451068A8160E00E94DE06A9
:1009A0008C8160E00E94DE068B818F3F19F060E051
:1009B0000E94DE066D8564FD1DC0CE0163E00E94CD
:1009C0003E0484E991E10E945106CE0163E00E9459
:1009D0003E0484E991E10E945106CE0163E00E9449
:1009E0003E0486E990E00E945106CE0162E00E943A
:1009F0003E0416C06062CE010E94A10484E991E128
:100A00000E9451066D856062CE010E94A10486E9B4
:100A100090E00E9451066D856062CE010E94A104A3
:100A20006D856062CE010E94A10484E08E87CE01B4
:100A30000E94A504CE010E94AF0482E08F87CE0100
:100A400066E00E94A104DF91CF9108956F927F929A
:100A50008F92AF92CF92EF920F931F93DF93CF932A
:100A6000CDB7DEB73C01162F842FF30142832383D9
:100A70000483E582C682A78280869D8591879E85B4
:100A800092879F8593879889948761E00E94B80632
:100A9000F30183818F3F19F061E00E94B806F301F2
:100AA000848161E00E94B806112319F0F3011586D4
:100AB00003C080E1F3018587C30160E141E020E0EC
:100AC0000E94B704CF91DF911F910F91EF90CF90CB
:100AD000AF908F907F906F9008958F92AF92CF924A
:100AE000EF920F931F93CF93DF93DC01362F542F98
:100AF000722F102FAE2C8C2C89E191E011969C93D3
:100B00008E9300D000D0EDB7FEB73196CDB7DEB7EB
:100B10001982118212821382CD0161E0432F2FEFDF
:100B2000052FE72EC12E0E9426050F900F900F90E3
:100B30000F90DF91CF911F910F91EF90CF90AF90D9
:100B40008F9008951F920F920FB60F9211242F933A
:100B50003F938F939F93AF93BF938091AD019091FB
:100B6000AE01A091AF01B091B0013091B1010196F9
:100B7000A11DB11D232F2D5F2D3720F02D5701967C
:100B8000A11DB11D2093B1018093AD019093AE01E1
:100B9000A093AF01B093B0018091A9019091AA01F7
:100BA000A091AB01B091AC010196A11DB11D809344
:100BB000A9019093AA01A093AB01B093AC01BF919E
:100BC000AF919F918F913F912F910F900FBE0F90FA
:100BD0001F9018958FB7F8942091AD013091AE0118
:100BE0004091AF015091B0018FBFB901CA01089582
:100BF0009B01AC017FB7F8948091A9019091AA0163
:100C0000A091AB01B091AC0166B5A89B05C06F3F48
:100C100019F00196A11DB11D7FBFBA2FA92F982FE2
:100C20008827860F911DA11DB11D62E0880F991FB5
:100C3000AA1FBB1F6A95D1F7BC012DC0FFB7F8945E
:100C40008091A9019091AA01A091AB01B091AC0152
:100C5000E6B5A89B05C0EF3F19F00196A11DB11D97
:100C6000FFBFBA2FA92F982F88278E0F911DA11D86
:100C7000B11DE2E0880F991FAA1FBB1FEA95D1F7AB
:100C8000861B970B885E9340C8F22150304040404D
:100C9000504068517C4F211531054105510571F6D1
:100CA0000895019739F0880F991F880F991F0297AF
:100CB0000197F1F70895789484B5826084BD84B576
:100CC000816084BD85B5826085BD85B5816085BD47
:100CD000EEE6F0E0808181608083E1E8F0E0108260
:100CE000808182608083808181608083E0E8F0E0A1
:100CF000808181608083E1EBF0E08081846080838B
:100D0000E0EBF0E0808181608083EAE7F0E08081C1
:100D10008460808380818260808380818160808321
:100D20008081806880831092C1000895982F8E3052
:100D300008F09E509770809114018295880F880F5B
:100D4000807C892B80937C0080917A0080648093E2
:100D50007A0080917A0086FDFCCF20917800409146
:100D60007900942F80E030E0282B392BC9010895B9
:100D7000482F50E0CA0186569F4FFC0124914A57E4
:100D80005F4FFA0184918823C1F0E82FF0E0EE0F65
:100D9000FF1FE859FF4FA591B491662341F49FB717
:100DA000F8948C91209582238C939FBF08959FB7D0
:100DB000F8948C91822B8C939FBF0895482F50E01C
:100DC000CA0182559F4FFC012491CA0186569F4F4C
:100DD000FC0134914A575F4FFA019491992309F429
:100DE00044C0222351F1233071F0243028F4213003
:100DF000A1F0223011F514C02630B1F02730C1F037
:100E00002430D9F404C0809180008F7703C0809192
:100E100080008F7D8093800010C084B58F7702C0E2
:100E200084B58F7D84BD09C08091B0008F7703C0E9
:100E30008091B0008F7D8093B000E92FF0E0EE0F3D
:100E4000FF1FEE58FF4FA591B491662341F49FB761
:100E5000F8948C91309583238C939FBF08959FB70E
:100E6000F8948C91832B8C939FBF08951F920F92BF
:100E70000FB60F9211242F933F934F938F939F930D
:100E8000EF93FF934091C600E0913202F09133025C
:100E900031969F012F773070319780913402909175
:100EA00035022817390739F0EE54FE4F408330934E
:100EB000330220933202FF91EF919F918F914F91D6
:100EC0003F912F910F900FBE0F901F901895CF93C9
:100ED000DF93EC019A01AB01E885F985203081EEC2
:100EE000380780E0480780E0580709F449C081E0EE
:100EF00090E00A8802C0880F991F0A94E2F7808365
:100F000060E079E08DE390E00E94F40C21503040E5
:100F100040405040CA01B90122E030E040E050E0DA
:100F20000E94F40CEC81FD813083EE81FF812083EF
:100F3000EA85FB85208141E050E0CA010E8402C0B1
:100F4000880F991F0A94E2F7282B2083EA85FB85F6
:100F50002081CA010F8402C0880F991F0A94E2F70A
:100F6000282B2083EA85FB858081088802C0440FF6
:100F7000551F0A94E2F7842B8083DF91CF91089567
:100F8000108220E130E0CECFDC011296ED91FC9191
:100F90001397E058FF4F2191319180819181281B57
:100FA000390B2F773070C9010895DC011296ED914D
:100FB000FC911397EE57FF4F2081318192918291DE
:100FC000E058F0408217930719F42FEF3FEF05C068
:100FD000E20FF31F8081282F30E0C9010895DC0162
:100FE0001296ED91FC911397DF01AE57BF4F2D91F3
:100FF0003C911197E058FF4F80819181E058F0407B
:101000008217930719F42FEF3FEF0BC0E20FF31F86
:1010100080812F5F3F4F2F7730702D933C93282F87
:1010200030E0C9010895DC011296ED91FC9113970F
:10103000EE57FF4F80819181929382930895FC0136
:10104000A085B18521898C9190E0022E02C09595F2
:1010500087950A94E2F780FFF6CF0484F585E02DAA
:101060006083089583E291E0909337028093360283
:1010700082EB91E0909339028093380285EC90E006
:1010800090933B0280933A0284EC90E090933D026F
:1010900080933C0280EC90E090933F0280933E026C
:1010A00081EC90E0909341028093400286EC90E0C6
:1010B000909343028093420284E08093440283E051
:1010C0008093450287E08093460285E08093470243
:1010D00081E08093480208950E945B060E94D70336
:1010E0000E94CC00FDCF0F931F93CF93DF938C0111
:1010F000EB0109C02196D801ED91FC910190F0819E
:10110000E02DC801099568816623A1F7DF91CF9191
:101110001F910F910895EF92FF920F931F93CF931A
:10112000DF938C017B01EA010CC0D7016D917D0139
:10113000D801ED91FC910190F081E02DC801099555
:101140002197209791F7DF91CF911F910F91FF90F9
:10115000EF900895DC01ED91FC910280F381E02D88
:10116000099508952F923F924F925F926F927F92CE
:101170008F929F92AF92BF92CF92DF92EF92FF92A7
:101180000F931F93DF93CF93CDB7DEB7A0970FB622
:10119000F894DEBF0FBECDBF1C016A017B01411573
:1011A00051056105710549F440E350E060E070E0ED
:1011B00020E030E00E945B0956C088249924540145
:1011C000422E55246624772401E010E00C0F1D1FE9
:1011D000080D191DC701B601A30192010E94D20C8E
:1011E000F80160830894811C911CA11CB11CC701EB
:1011F000B601A30192010E94D20CC901DA016C016F
:101200007D01C114D104E104F104F1F681E0E82E7E
:10121000F12CEC0EFD1EE80CF91C3E010894611C3B
:10122000711CD501C4010197A109B1096C01C8184D
:10123000D90816C0F601EE0DFF1D40814A3010F4AA
:10124000405D01C0495C552747FD5095652F752FBE
:10125000C10120E030E00E945B090894E108F10838
:101260006E147F0439F7A0960FB6F894DEBF0FBE58
:10127000CDBFCF91DF911F910F91FF90EF90DF9045
:10128000CF90BF90AF909F908F907F906F905F9026
:101290004F903F902F900895DC012115310541F4C6
:1012A000ED91FC910190F081E02D642F0995089556
:1012B0000E94B2080895EF92FF920F931F93CF936D
:1012C000DF93EC017A018B012115310541F4E881AE
:1012D000F9810190F081E02D642F09951BC02A301F
:1012E0003105B1F477FF10C04DE250E060E070E0EE
:1012F00020E030E00E945B0910950095F094E094A6
:10130000E11CF11C011D111DCE01B801A7012AE04D
:101310000E94B208DF91CF911F910F91FF90EF9043
:101320000895EF92FF920F931F93E62E9A01FF24E8
:10133000E7FCF0940F2D1F2DB801A7010E945B0957
:101340001F910F91FF90EF9008950F931F938C01C1
:101350004DE050E060E070E020E030E00E945B098A
:10136000C8014AE050E060E070E020E030E00E9418
:101370005B091F910F9108959F92AF92BF92CF92F8
:10138000DF92EF92FF920F931F93CF93DF93EC01C5
:101390007A018B01922ECB01BA0120E030E040E0CF
:1013A00050E00E94BB0A88236CF4CE014DE250E06D
:1013B00060E070E020E030E00E945B0917FB1095D0
:1013C00017F9109520E030E040E05FE3AA240BC05D
:1013D000CA01B90120E030E040E251E40E94BF0AB6
:1013E0009B01AC01A394A91498F3C801B7010E9412
:1013F000570A5B016C010E942C0B7B018C01CE0112
:10140000B801A7012AE030E00E944C09992029F098
:10141000CE0160E071E00E94AA08C801B7010E94F5
:10142000580B9B01AC01C601B5010E94560A22C0AF
:1014300020E030E040E251E40E940A0C7B018C0184
:101440000E94270B5B016C01CC24B7FCC094DC2C00
:10145000CE01B601A5012AE030E00E945B09C60179
:10146000B5010E945A0B9B01AC01C801B7010E9453
:10147000560A9A949920E1F6DF91CF911F910F912E
:10148000FF90EF90DF90CF90BF90AF909F90089526
:101490000E94BC0908950F931F938C010E94BC0900
:1014A000C8010E94A5091F910F9108955058BB27AC
:1014B000AA270ED075C166D130F06BD120F031F47F
:1014C0009F3F11F41EF45BC10EF4E095E7FB51C1A0
:1014D000E92F77D180F3BA1762077307840795075E
:1014E00018F071F49EF58FC10EF4E0950B2EBA2F13
:1014F000A02D0B01B90190010C01CA01A00111241A
:10150000FF27591B99F0593F50F4503E68F11A16C5
:10151000F040A22F232F342F4427585FF3CF469556
:1015200037952795A795F0405395C9F77EF41F1678
:10153000BA0B620B730B840BBAF09150A1F0FF0F42
:10154000BB1F661F771F881FC2F70EC0BA0F621F2E
:10155000731F841F48F4879577956795B795F7951E
:101560009E3F08F0B3CF9395880F08F09927EE0FB0
:10157000979587950895D9D008F481E008950CD007
:101580000FC107D140F0FED030F021F45F3F19F0D9
:10159000F0C0511139C1F3C014D198F39923C9F3A4
:1015A0005523B1F3951B550BBB27AA276217730769
:1015B000840738F09F5F5F4F220F331F441FAA1F1D
:1015C000A9F333D00E2E3AF0E0E830D091505040DD
:1015D000E695001CCAF729D0FE2F27D0660F771F8B
:1015E000881FBB1F261737074807AB07B0E809F06D
:1015F000BB0B802DBF01FF2793585F4F2AF09E3F02
:10160000510568F0B6C000C15F3FECF3983EDCF3D3
:10161000869577956795B795F7959F5FC9F7880F7A
:10162000911D9695879597F90895E1E0660F771FCC
:10163000881FBB1F621773078407BA0720F0621B5D
:10164000730B840BBA0BEE1F88F7E095089504D056
:101650006894B111D9C00895BCD088F09F5790F01C
:10166000B92F9927B751A0F0D1F0660F771F881FC7
:10167000991F1AF0BA95C9F712C0B13081F0C3D0E2
:10168000B1E00895C0C0672F782F8827B85F39F080
:10169000B93FCCF3869577956795B395D9F73EF426
:1016A00090958095709561957F4F8F4F9F4F0895CE
:1016B000E89409C097FB3EF49095809570956195EC
:1016C0007F4F8F4F9F4F9923A9F0F92F96E9BB27A2
:1016D0009395F695879577956795B795F111F8CF1E
:1016E000FAF4BB0F11F460FF1BC06F5F7F4F8F4F89
:1016F0009F4F16C0882311F096E911C0772321F07F
:101700009EE8872F762F05C0662371F096E8862F16
:1017100070E060E02AF09A95660F771F881FDAF76D
:10172000880F9695879597F90895990F0008550F9A
:10173000AA0BE0E8FEEF16161706E807F907C0F057
:1017400012161306E407F50798F0621B730B840B5F
:10175000950B39F40A2661F0232B242B252B21F439
:1017600008950A2609F4A140A6958FEF811D811DD9
:10177000089597F99F6780E870E060E008959FEF13
:1017800080EC089500240A94161617061806090618
:10179000089500240A9412161306140605060895E7
:1017A000092E0394000C11F4882352F0BB0F40F46F
:1017B000BF2B11F460FF04C06F5F7F4F8F4F9F4FAF
:1017C000089557FD9058440F551F59F05F3F71F031
:1017D0004795880F97FB991F61F09F3F79F0879598
:1017E0000895121613061406551FF2CF4695F1DF21
:1017F00008C0161617061806991FF1CF86957105B1
:10180000610508940895E894BB2766277727CB01E4
:1018100097F908950BD0C4CFB5DF28F0BADF18F0E0
:10182000952309F0A6CFABCF1124EECFCADFA0F3EA
:10183000959FD1F3950F50E0551F629FF001729F65
:10184000BB27F00DB11D639FAA27F00DB11DAA1F84
:10185000649F6627B00DA11D661F829F2227B00DD1
:10186000A11D621F739FB00DA11D621F839FA00D5C
:10187000611D221F749F3327A00D611D231F849FAC
:10188000600D211D822F762F6A2F11249F57504003
:101890008AF0E1F088234AF0EE0FFF1FBB1F661F9E
:1018A000771F881F91505040A9F79E3F510570F057
:1018B00060CFAACF5F3FECF3983EDCF38695779537
:1018C0006795B795F795E7959F5FC1F7FE2B880F52
:1018D000911D9695879597F9089511F40EF44FCFC1
:1018E0004AC077DFD0F39923D9F3CEF39F57550B36
:1018F00087FF51D056959795B0E020F4660F771F7B
:10190000881FBB1F1F930F9300249001A00180012B
:10191000F001A0E80E0F1F1F0A1E511D601B710B66
:101920008009B50B48F4600F711F801DB51F0E1B99
:101930001F0B0A0A510907C02E0F3F1F4A1F0E0F27
:101940001F1F0A1E511D660F771F881FBB1FA695FC
:10195000F795E795F8F60617170708065B07211DA8
:10196000311D411D0F911F91B901842F9158880F8E
:101970009695879508959F3F49F0915028F4869554
:1019800077956795B7959F5F80389F4F880F96959D
:10199000879597F9089591505040660F771F881FDB
:1019A000D2F70895A1E21A2EAA1BBB1BFD010DC0A0
:1019B000AA1FBB1FEE1FFF1FA217B307E407F507FF
:1019C00020F0A21BB30BE40BF50B661F771F881FDB
:1019D000991F1A9469F760957095809590959B0171
:1019E000AC01BD01CF01089597FB092E05260ED04D
:1019F00057FD04D0D7DF0AD0001C38F4509540952D
:101A0000309521953F4F4F4F5F4F0895F6F79095D2
:101A10008095709561957F4F8F4F9F4F0895EE0F82
:0E1A2000FF1F0590F491E02D0994F894FFCF7C
:101A2E002E00B80B020001000000803F0000803F36
:101A3E003333134001000000009D0473088B08002F
:101A4E000000001F0873088B08C407EF07D50713A3
:021A5E0008007E
:00000001FF
